:100000000C946C020C9494020C9494020C94940240
:100010000C9494020C9494020C9494020C94940208
:100020000C9494020C9494020C9494020C94D804B2
:100030000C9494020C9494020C9494020C949402E8
:100040000C9452040C9494020C9494020C94940218
:100050000C9494020C9494020C9494020C949402C8
:100060000C9494020C9494020101FF030101F70324
:100070006C00680000000000240027002A00000037
:100080000000250028002B000500893008023802F6
:100090004978681400002020202020476F6F6420DA
:1000A0006A6F622100175344001613780016131468
:1000B000001510200015201000540A03E181867FEE
:1000C0003E186D830F0F0E0183866033186DC319C0
:1000D0008F1803C38E6033186DE330CF1803C39EAF
:1000E000603630CDE360CF3006C79E7E3E30CDB364
:1000F00060CF300CC6F6603330D9B660CF33CFCC8A
:10010000F66061B0DB1E60CF30D86CE6C061B0DB5A
:100110001E618F19986CC6C063B19B0E330F0FB070
:1001200078C6FF7E1F1B061E0F40246FFFFFFFFFD8
:10013000FFFFFF6FFFFFFFFFFFFFFF688200A000D0
:100140002A20036EEEBEBEFBEAEBFF60088A002A9F
:10015000200A8B7BAEFBAFAFAEEEBB60A02AA20A3B
:1001600008200B7BBEEAEFFAEFAEEB6AA00028286E
:10017000A2A2836AFFBAFBEEBEFFBB6002AA000226
:1001800080280B7BFEEFAEFABAAEFB608000A8823F
:100190008A822B7BBEABFFFFFBBFEF6008ABFFFF8C
:1001A000FA000B7AEEBB77FFFBAEEB62228B24E307
:1001B000B8A2237AEAFF567B5EEEAB622A835577BC
:1001C000388AAB7BFFFB74639BBBAB6000A3FFFF74
:1001D000F880AB7BFAAFFFFFFBFAFB602220A02A7E
:1001E000200A2B6FBBFFBFABBFBAEB622A00002A0D
:1001F00080AA236AAEFBBEEAEFEFFF6A800A08001E
:100200000288036FEEBFFAEEEEBEAB6022880A8270
:100210008000AB7BEBBBFBABEEEFAF6888800AA83E
:100220002222A36EFEEAEEFBBFAAAF60028A202262
:1002300000A8A37FFFFFFFFFFFFFFB7FFFFFFFFF84
:10024000FFFFFB0000000000000000000500380177
:1002500068010000F6E8DBCFC3B8AEA49B928A82A7
:100260007B746E68625C57524E4945413E3A373462
:10027000312E2C29272523210A0A153A49676E6F4A
:100280007265006D560A0A504C454153452054553D
:10029000524E204F464620004C4F57204241545466
:1002A00045525921200003053F213F1208120A1030
:1002B0000A0E1C0E0C1E0C141A14161F161E131EEA
:1002C0001E1B1E1E1F1E3F213F3A2F3A173D173F90
:1002D000213F181F02040A041F0E04040E1F0A1FE8
:1002E0000A0E0E1F04110E2E252E2F2A2E26292926
:1002F000021F02081F08150E04040E150E15151B0B
:10030000151B040604040C04000000001700030081
:10031000031F0A1F16371A1904130A153A0003009F
:10032000000E11110E000A040A040E04003000042D
:1003300004040010001804031F111F121F101D15C4
:100340001711151F07041F17151D1F151D01011F6C
:100350001F151F17151F000A00003200040A110A9A
:100360000A0A110A040115020E11171E051E1F1597
:100370000A0E110A1F110E1F15111F05010E111D66
:100380001F041F111F1108100F1F041B1F10101F27
:10039000061F1E040F0E110E1F09060E112E1F053B
:1003A0001A121509011F011F101F0F180F1F0C1F14
:1003B0001B041B031C03191513001F110304181140
:1003C0001F000201022020200001020C121E1F1239
:1003D0000C0C12120C121F0C1A14041E05242A1ED7
:1003E0001F021C141D1020201D1F0814111F101E99
:1003F000041E1E021C0C120C3E0A040C123E1E04AB
:100400000214160A020F120E101E0E100E1E081EE7
:10041000120C1226281E322A26041E21001F00213B
:100420001E040102013F213F172B152010204C4FC5
:100430004144455200172B16201314000A4E6F201A
:1004400053442063617264206F720A6E6F204C4FB8
:10045000414445522E4845580A0A153A4578697470
:10046000001D20466C617368696E670A20206C6FFE
:10047000616465722E2E2E0A0A444F4E2754205472
:1004800055524E204F464621000000000023002612
:100490000029000404040404040404020202020209
:1004A0000203030303030301020408102040800138
:1004B00002040810200102040810200000000800B7
:1004C00002010000030407000000000000000045D6
:1004D0000068010000004B1811241FBECFEFD8E0C8
:1004E000DEBFCDBF11E0A0E0B1E0E0E2F5E302C085
:1004F00005900D92AC31B107D9F727E0ACE1B1E03E
:1005000001C01D92A53AB207E1F712E0CCE6D2E0B5
:1005100004C02197FE010E94831ACB36D107C9F788
:100520000E9488120C948E1A0C940000CF92DF92D5
:10053000EF92FF920F931F93CF93DF936C017A0199
:100540008B01C0E0D0E0CE15DF0589F0D8016D91B8
:100550008D01D601ED91FC910190F081E02DC60155
:100560000995892B11F47E0102C02196ECCFC701B9
:10057000DF91CF911F910F91FF90EF90DF90CF907F
:100580000895BC0190910E059E31D8F4E2EDF4E09F
:1005900040E050E0292F30E04217530744F4A19186
:1005A000B191A617B70769F04F5F5F4FF5CF220FE4
:1005B000331FF901EE52FB4F718360839F5F90936D
:1005C0000E050895089580E090E008950E94891A2C
:1005D000833081F028F4813099F08230A1F00895C1
:1005E0008730A9F08830B9F08430D1F48091800050
:1005F0008F7D03C0809180008F7780938000089565
:1006000084B58F7702C084B58F7D84BD08958091B5
:10061000B0008F7703C08091B0008F7D8093B000D1
:1006200008951F93CF93DF93282F30E0F901E5540D
:10063000FB4F8491F901E955FB4FD491F901ED5637
:10064000FB4FC491CC23C9F0162F81110E94E80200
:10065000EC2FF0E0EE0FFF1FE258FF4FA591B49191
:100660008FB7F894111105C09C91ED2FE095E92307
:1006700002C0EC91ED2BEC938FBFDF91CF911F91D6
:100680000895CF93DF9390E0FC01E955FB4F24914F
:10069000FC01ED56FB4F8491882361F190E0880FB7
:1006A000991FFC01EC58FF4FC591D491FC01E25811
:1006B000FF4FA591B491611109C09FB7F89488814B
:1006C000209582238883EC912E230BC0623061F445
:1006D0009FB7F8943881822F809583238883EC918B
:1006E0002E2B2C939FBF06C08FB7F894E8812E2B3A
:1006F00028838FBFDF91CF9108951F93CF93DF930E
:10070000182FEB0161E00E944103209711F460E093
:1007100004C0CF3FD10539F461E0812FDF91CF9143
:100720001F910C941103E12FF0E0E554FB4FE4918D
:10073000E330F9F048F4E130B9F0E230A1F584B5E6
:10074000806284BDC8BD34C0E730E9F0E83019F1FB
:10075000E43049F580918000806280938000D093DE
:100760008B00C0938A0024C084B5806884BDC7BD57
:100770001FC080918000806880938000D0938900A2
:10078000C093880015C08091B00080688093B0004D
:10079000C093B3000DC08091B00080628093B00020
:1007A000C093B40005C0C038D1050CF0B5CFAFCFB1
:1007B000DF91CF911F9108958E3008F08E50877091
:1007C000806480937C0080917A00806480937A00BA
:1007D00080917A0086FDFCCF80917800209179008D
:1007E00090E0922B08953FB7F89480911105909175
:1007F0001205A0911305B091140526B5A89B05C05C
:100800002F3F19F00196A11DB11D3FBFBA2FA92F8F
:10081000982F8827820F911DA11DB11DBC01CD010C
:1008200042E0660F771F881F991F4A95D1F70895F8
:100830008F929F92AF92BF92CF92DF92EF92FF92F0
:100840006B017C010E94F3034B015C01C114D104D4
:10085000E104F104F1F00E94F303DC01CB018819FB
:100860009909AA09BB09883E9340A105B10570F317
:1008700021E0C21AD108E108F10888EE880E83E071
:10088000981EA11CB11CC114D104E104F10419F794
:10089000DDCFFF90EF90DF90CF90BF90AF909F9013
:1008A0008F9008951F920F920FB60F9211242F93DD
:1008B0003F938F939F93AF93BF9380911705909130
:1008C0001805A0911905B0911A053091100523E083
:1008D000230F2D3720F40196A11DB11D05C026E878
:1008E000230F0296A11DB11D2093100580931705BB
:1008F00090931805A0931905B0931A0580911105DE
:1009000090911205A0911305B09114050196A11DB7
:10091000B11D8093110590931205A0931305B09318
:100920001405BF91AF919F918F913F912F910F909F
:100930000FBE0F901F90189580911B07882319F008
:1009400080911D0701C080E08093B4000895CF938B
:10095000DF93EC011F8A1D8A1CA21BA2188E109225
:100960001D0710921C0710921B070E949C048CE428
:1009700092E09E878D871B8A1A8A81E0898389E0AD
:100980008E8B198E1B8E1D8EDF91CF910895FC01E9
:1009900061110DC0178A158A14A213A2108E10922D
:1009A0001D0710921C0710921B070C949C040895BD
:1009B0001F920F920FB60F9211242F933F934F93D4
:1009C0005F936F937F938F939F93AF93BF93EF93B7
:1009D000FF9360911C07662321F180910F058F5FC3
:1009E00080930F05909115058917D8F090911B07FA
:1009F00081E0892780931B0710920F0580911605CF
:100A0000882369F08091000193E4899F802D11244F
:100A1000895B809300010E944F1A90931D070E94EA
:100A20009C04FF91EF91BF91AF919F918F917F9126
:100A30006F915F914F913F912F910F900FBE0F904B
:100A40001F901895FC01643508F053C0403308F03E
:100A500050C090A1742F759575957595262F062E0B
:100A6000000C330B542F57709230A1F4F901E55E5E
:100A7000FA4F84E57802E00DF11D1124808190E0A9
:100A8000052E02C0959587950A94E2F78095982FD8
:100A900091700AC0933041F4848581704627409557
:100AA0004170841303C014C0911112C084E5780210
:100AB000200D311D1124F901E55EFA4F81E090E02F
:100AC00001C0880F5A95EAF780959081892310C05C
:100AD00084E57802200D311D1124F901E55EFA4FFD
:100AE00081E090E001C0880F5A95EAF79081892B48
:100AF00080830895DF92EF92FF920F931F93CF931D
:100B0000DF931F92CDB7DEB78C01D62EF42EE12CE9
:100B1000E21654F46E2D6D0D4F2DC80129830E94ED
:100B20002205E3942981F4CF0F90DF91CF911F919B
:100B30000F91FF90EF90DF900895DF92EF92FF9278
:100B40000F931F93CF93DF937C01D62FD22EC42F08
:100B5000002E000C110B040F111D47FD1A954C2F90
:100B60000C2E000C550B4017510744F42D2D4C2F23
:100B70006D2FC7010E947A05CF5FF1CFDF91CF9132
:100B80001F910F91FF90EF90DF9008956F927F92E9
:100B90008F929F92AF92BF92CF92DF92EF92FF928D
:100BA0000F931F93CF93DF93EC016A3019F42D81DB
:100BB0009885A1C06D3009F4A4C01885BA84D98481
:100BC00088A083E58D150CF47FC08FE28B150CF4A3
:100BD0007BC08C8190E00197189F9001199F300D88
:100BE0001124C9018D0D911DD7FC9A95181619066F
:100BF0000CF06AC08D81819FC00111248B0D911D65
:100C0000B7FC9A95181619060CF05EC09D2CCD2CD9
:100C1000E62EF12CEC2DED190E2E000CFF0B8C8125
:100C200090E0E817F9070CF04EC00197E817F907B4
:100C300079F0E89E9001E99E300DF89E300D112468
:100C4000E20FF31F8E8D9F8DE80FF91F749001C086
:100C5000712C6B2CAB2C2A2D2B19022E000C330B74
:100C60008D8190E0281739075CF570FE10C01130B7
:100C700031F44A2D6C2DCE010E9422051DC0012F9A
:100C8000212F462D692DCE010E949D0515C089A1F9
:100C900098A1891789F088A3113031F44A2D6C2D61
:100CA000CE010E94220507C0012F212F462D692D5C
:100CB000CE010E949D0588A27694A394610ECBCFAD
:100CC000C394910EA7CF88A228853C818985329F45
:100CD000800D112489879F81992399F0082E000C9B
:100CE000990B44E550E0239F4019510911244817FE
:100CF00059073CF49D818A85299F800D11248A879C
:100D0000198681E090E0DF91CF911F910F91FF90C4
:100D1000EF90DF90CF90BF90AF909F908F907F909B
:100D20006F900895DF92EF92FF920F931F93CF93EE
:100D3000DF931F92CDB7DEB78C01D62EF42EE12CB7
:100D4000E21654F44E2D4F0D6D2DC80129830E94DB
:100D50002205E3942981F4CF0F90DF91CF911F9169
:100D60000F91FF90EF90DF9008953091CA0450E00A
:100D7000639F400D511D1124FA0133E0F595E7956D
:100D80003A95E1F747705527E80FF91F222369F0DC
:100D900027E030E0241B350B81E090E001C0880F94
:100DA0002A95EAF79081892B0DC027E030E0241BBB
:100DB000350B81E090E001C0880F2A95EAF7809515
:100DC00090818923808308952091CA0450E0629F16
:100DD000400D511D11249A0163E0359527956A95C0
:100DE000E1F7820F931FFC01808190E040955095C0
:100DF0004770552702C0959587954A95E2F781700F
:100E00000895EF92FF920F931F93CF93DF93182FC4
:100E1000062F20E0462F682F85E592E00E94B50658
:100E2000E02EF12C8091CA0490E00297C12FD0E00F
:100E3000E816F9064CF441E0400F612F85E592E099
:100E40000E94E406811133C0002349F04FEF400FA8
:100E5000612F85E592E00E94E406811132C0809105
:100E6000C70490E00297C817D9074CF4402F61E0FF
:100E7000610F85E592E00E94E40681112CC01123E8
:100E800099F16FEF610F402F85E592E00E94E40633
:100E9000882351F121979C2F88278E0D9F1DDF916C
:100EA000CF911F910F91FF90EF900C94C1029C2F56
:100EB000882797012F5F3F4F820F931F0E94C10227
:100EC000C3CF9C2F8827970121503109820F931F90
:100ED0000E94C102C4CFCE010196982F88278E0DA3
:100EE0009F1D0E94C102CBCFDF91CF911F910F9127
:100EF000FF90EF9008954F925F926F927F928F9242
:100F00009F92AF92BF92CF92DF92EF92FF920F9398
:100F10001F93CF93DF938093CA046093C704EEE8D6
:100F2000F3E08FEF94E0E73CF90711F08193FACFFB
:100F3000ECE1F1E08FEF92E0E535F90711F08193F4
:100F4000FACFE5E5F2E08FEF93E0EE38F90711F024
:100F50008193FACF10920E0560E080E00E940107B5
:100F600034E0432E512C612C712CC0910E05CC2302
:100F700009F48EC00E94A4182C2F30E040E050E00D
:100F80000E94B218660F771FDB01AE52BB4F0D9166
:100F90001C91119780910E05E82FF0E0EE0FFF1FD6
:100FA000E053FB4F208131812D933C9381508093FE
:100FB0000E05C12FDD27EC2EF02E88248A948C0E8E
:100FC000DD24D394DC0E99249A94900E5801BB240E
:100FD000CC24C394C00E0E94A418A30192010E94C5
:100FE000B2186130710581059105F1F02CF4672B81
:100FF000682B692B61F0EFCF623071058105910597
:1010000029F1633071058105910571F1E4CFFF206D
:1010100011F3492D6E2D85E592E00E94E4068111C1
:10102000DACF20E0402F6DC08091CA0490E0029793
:10103000A816B90684F64C2D6E2D85E592E00E9427
:10104000E4068111C8CF20E04C2D5BC0209719F237
:101050004F2D682D85E592E00E94E4068111BBCFFB
:1010600020E0402F6C2F51C08091C70490E0029780
:10107000C817D9070CF0AFCF4F2D6D2D85E592E045
:101080000E94E4068111A7CF20E0402F6D2D3DC0C6
:1010900020E040E060E08EE893E00E94B5064091D9
:1010A000CA0442506091C704615020E08EE893E08A
:1010B0000E94B5061092CE041092CD041092D00476
:1010C0001092CF041092C9041092C8041092CC045C
:1010D0001092CB0421E040E060E085E592E0DF91F2
:1010E000CF911F910F91FF90EF90DF90CF90BF9025
:1010F000AF909F908F907F906F905F904F900C94E7
:10110000B5066C2F8CE191E002C08EE893E00E945E
:10111000B506602F8C2F0E94010780910E0581116A
:1011200024CFC0E08C2F90E02091C70430E0215004
:101130003109821793070CF018CFD0E02D2F30E043
:101140008091CA0490E001972817390774F44D2F55
:101150006C2F85E592E00E94E406811104C06D2F9A
:101160008C2F0E940107DF5FE9CFCF5FDBCF8F922B
:101170009F92AF92BF92CF92DF92EF92FF920F9326
:101180001F93CF93DF9380918E07882309F4B8C013
:1011900081E0809374071092730710927207109287
:1011A000360780938C0780938D07CBE4D2E01CE058
:1011B0000E94D6098823E1F3FE018491882319F067
:1011C0000091710701C000E069EB70E080E00E94CF
:1011D0008B1169E271E08CE0800F0E948B111092FC
:1011E0007507109376078BE492E00E94150F8091AB
:1011F0007007982F990F890F81958D5A80937507E5
:1012000080917107982F990F890F8195835D809345
:10121000760780918F0784FF03C085EB90E002C0C2
:1012200081EB90E00E94360F80917007982F990F04
:10123000890F81958D5A80937507809176078F5F0E
:101240008093760780914807882319F08DEA90E013
:1012500002C089EA90E00E94360F80917007982FB3
:10126000990F890F81958D5A809375078091760724
:101270008F5F8093760785EA90E00E94360F809119
:1012800034078130A1F4809148078F5F609149074E
:1012900087FD09C0082E000C990B70E06F5F7F4F2F
:1012A0000E945B1A682F609348070E943B0E809152
:1012B00033078130B9F080918E07482F50E060E00D
:1012C00070E0C0908F07D0909007E0909107F09069
:1012D0009207C416D506E606F70608F45FC08F3FEE
:1012E00009F45CC08FEF80938E0760E083E497E0A1
:1012F0000E94C7041092440783E497E00E94A70469
:1013000010923607C0903807D0903907C094D09417
:10131000E12CF12C0E94F3034B015C010E94F303CA
:10132000A501940120953095409550956095709554
:10133000809590950E943F1A9B01AC01C701B601B0
:101340000E943F1A4B015C0180911F07909120077A
:101350006C01E12CF12C0E94F303C60ED71EE81E8F
:10136000F91EC701B601680D791D8A1D9B1D611507
:1013700071058105910511F00E94A9186AE08AE0C3
:10138000DF91CF911F910F91FF90EF90DF90CF9061
:10139000BF90AF909F908F900C947B078091350702
:1013A000813009F005CF0E94440F02CF4F925F9227
:1013B0006F927F928F929F92AF92BF92CF92DF9265
:1013C000EF92FF920F931F93CF93DF9300D000D043
:1013D0001F92CDB7DEB740919E0750919F07609155
:1013E000A0077091A1072FB7F894809117059091ED
:1013F0001805A0911905B0911A052FBF481B590B6C
:101400006A0B7B0B80919D0790E0A0E0B0E000911B
:10141000990710919A0720919B0730919C07841798
:101420009507A607B70730F4011511052105310509
:1014300009F027C3012B022B032B09F020C3809155
:10144000350781508E3F08F580913407813011F5C2
:10145000809148078F5F6091490787FD09C0082E7A
:10146000000C990B70E06F5F7F4F0E945B1A682F32
:101470006093480785E394E09093A3078093A207C5
:1014800088E48093A4070E943B0E80913507815029
:101490008E3F70F480913307813009F09EC388E25B
:1014A00094E09093A3078093A20788E48093A40715
:1014B00080E00E94790F80914407882309F4ADC031
:1014C000809158078111A9C08091500790915107D0
:1014D000E0915507F0915607EE0FFF1FE80FF91F37
:1014E000459154914115510501F52091540722234E
:1014F00031F01092560710925507FC0114C010925B
:10150000440780914307882341F080E00E94790FCF
:10151000E0915507F09156072FC060E083E497E013
:101520000E94C7047AC0459154919A013695279537
:101530003695279540FF51C0CA0116E096958795CC
:101540001A95E1F78F71952F9695969596959051EE
:101550002F70223071F1F8F4211117C08B3008F090
:101560008AE080935907E0915507F091560731962C
:10157000F0935607E0935507EE0FFF1F8091500739
:1015800090915107E80FF91FCECF213061F760E04D
:101590000E94E60FE8CF2330B1F0243021F72091EC
:1015A0004707829F802D11248093600790936107E5
:1015B000DACF20914707829F802D112480935C070A
:1015C00090935D07D0CF20914707829F802D1124F3
:1015D00080935E0790935F07C6CF2F7320935707C2
:1015E00080914707859F802D112480935807109282
:1015F0006807109267071092660781E080935A0788
:1016000080931B0710925B078091550790915607B6
:101610000196909356078093550780915A07882327
:1016200009F4F3C080915807811106C060E083E49B
:1016300097E00E94C704E9C08150809358078091C9
:101640006807811148C020916607309167072F5FB6
:101650003F4FC901880F991FE0916207F09163071E
:10166000E80FF91F65917491862F87708093690741
:10167000AB01E3E056954795EA95E1F7CA019695E7
:101680008795972F9695969590936A078F7390916B
:101690004707899F802D11248093680741704093EC
:1016A000160530936707209366078091640790E0E2
:1016B0002817390780F020916507222339F0821B13
:1016C0009109909367078093660705C060E083E403
:1016D00097E00E94C7048091680781508093680753
:1016E00080915B0721E0280F20935B07409157070B
:1016F00030916A07340F80914F07380F30934507B8
:1017000060915E07662371F070E0822F022E000C5C
:10171000990B0E945B1A80915F07869F300D112400
:10172000309345078091450790E0849664E270E02D
:101730000E945B1A80934507309159073093460702
:1017400060915C07662381F0062E000C770B822FD8
:10175000022E000C990B0E945B1A80915D07869FF8
:10176000300D112430934607609160076623A1F085
:10177000822F220F990B70E00E945B1ACB0162E06E
:1017800070E00E945B1A2091610790914607289FA4
:10179000900D112490934607809146074F3341F0F6
:1017A0008A300CF089E087FD80E08093460702C014
:1017B00010924607F894E0914507F0E0EC5AFD4F8F
:1017C000E491E09315053091460720916B073203B1
:1017D00090011124409169074203C001439F900D7D
:1017E00011240090480702C0880F991F0A94E2F75D
:1017F00097FF02C081589F4F880F892F881F990B30
:1018000080931C0780931D0778948091A4078823F8
:1018100009F486C08C3020F49CE0E92EE81A01C05F
:10182000E12CFF24F394F092740710928C0710922D
:101830008D07309171074DE2D42E1D2D131B1E0D07
:1018400003E0030F2EE4412F63E08CE697E03D8335
:101850000E949D053D810CEF030F1D5F202F41E08D
:10186000612F80E50E949F10202F42E0612F83E0CE
:101870000E949F10F0928C07F0928D0700917107E3
:10188000FD2CF01AFE0C2EE44F2D63E08CE697E061
:101890000E947A0513E0100F1F0D4FEF410F2EE449
:1018A00063E08CE697E00E947A05035033E0F30E84
:1018B000202F4F2D60E08CE697E00E949206202FAB
:1018C0004F2D63E58CE697E00E94920641E06F2D74
:1018D00083E00E94211042E06F2D80E50E942110DC
:1018E000145044E0612F80E50E94211048E0612FF0
:1018F00083E00E94211084E0809375078091710736
:10190000E81A8E2D815D809376078091A2079091D1
:10191000A3070E94150F8091A40781508093A4070C
:1019200080913A0790913B07892B09F480C011E020
:1019300010938C0710928D079091700785E5891B95
:10194000809375071092760780913707813009F4EC
:1019500051C030F090913607853008F063C05EC00A
:1019600060E083E497E00E94C7041092440710935C
:101970007407E6EAF2E0E491EF5FE0937007E7EACC
:10198000F2E0E491EF5FE093710788EA92E09093D0
:101990008B0780938A0710923B0710923A071092A8
:1019A000720718EA0E94D6098823E1F388E992E0D9
:1019B0000E94150F609138077091390780E090E020
:1019C0004AE00E94021183E892E00E94150F612F05
:1019D00062956F7070E080E090E04AE00E94021132
:1019E00088E792E00E94150F80913307813009F05B
:1019F000FAC01DC080918F0790919007A091910728
:101A0000B09192078F709927AA27BB270897A10545
:101A1000B10510F487E009C088E707C0992339F0C1
:101A20008B5F03C0992319F08FE20E9443110E943B
:101A3000D50E8091720781110EC088EF91E0EBE125
:101A4000F5E0DF019C011D9221503040E1F710923A
:101A50007507109276070E94F303609399077093BD
:101A60009A0780939B0790939C072091950730914C
:101A70009607621B730B709394076093930780E043
:101A8000CCC02FB7F8948091170590911805A091BC
:101A90001905B0911A052FBF20919D07820F911D46
:101AA000A11DB11D80939E0790939F07A093A0074F
:101AB000B093A10780918F0790919007A091910713
:101AC000B09192070196A11DB11D80938F0790934D
:101AD0009007A0939107B0939207109299071092E4
:101AE0009A0710929B0710929C070E94F303609341
:101AF0009507709396078093970790939807809126
:101B00001F07909120072FE0289F8001299F100D2B
:101B1000112485E10E94DC03800F911F24E096953B
:101B200087952A95E1F79093200780931F072091CE
:101B30001E07222309F44BC060912207262F30E0B4
:101B400040E050E029833A834B835C83C0902307B5
:101B5000D12CE12CF12C40912607509127074A0106
:101B6000A12CB12C20912407309125072901612C4B
:101B7000712C8217930728F09C014817590708F425
:101B80009A01C901A0E0B0E09C01AD01241935091A
:101B90004609570969817A818B819C816C197D097D
:101BA0008E099F090E943F1AA50194012419350945
:101BB000460957090E94B218C20ED31EE41EF51E34
:101BC000C09221076C2D70E085E00E947D030E9489
:101BD000620E0E944E1181E020C0893209F068CC6B
:101BE0000E94440F65CC115009F0DCCE60E070E03B
:101BF00085E00E947D0383B7817F846083BF83B7C4
:101C0000816083BF83B7816083BF889583B78E7FF0
:101C100083BF83B78E7F83BFC5CE0F900F900F9089
:101C20000F900F90DF91CF911F910F91FF90EF9048
:101C3000DF90CF90BF90AF909F908F907F906F90EC
:101C40005F904F900895BC01009791F0FC010190C6
:101C50000020E9F73197AF01481B590BE0916C0761
:101C6000F0916D070280F381E02D8CE697E00994F6
:101C700080E090E00895CF93DF93CEE1D7E01CAEF3
:101C80001AAE109267071092660710925B071092C7
:101C90001D0710921C0710921B070E949C048FECDA
:101CA00094E09BAB8AAB18AE1FAA81E08EA389E0BB
:101CB0008BAF10925C0710925E0710926007DF9165
:101CC000CF910895CF92DF92EF92FF920F931F93DF
:101CD000CF93DF93C8E2D7E00FE217E0FF24FA9436
:101CE00097E0E92EE00E62E088810E94410328819E
:101CF00030E0F901E554FB4F8491F901E955FB4FC0
:101D0000C490F901ED56FB4FD490DD2071F08111A4
:101D10000E94E802ED2DF0E0EE0FFF1FE757FB4FAA
:101D2000A591B491EC91EC21B1F4F80180818F5F21
:101D3000808360E088810E94410321960F5F1F4FDE
:101D4000E012D1CFDF91CF911F910F91FF90EF90D3
:101D5000DF90CF900895F8018081882371F3F80116
:101D60008F3F11F41082E5CFF082E3CFCF93C82FDD
:101D7000F89460E080917B070E94110380917C07BA
:101D800018161CF460E00E941103CEBD00000DB4D3
:101D900007FEFDCF8EB580917C0718161CF461E01C
:101DA0000E9411037894CF9108950F931F93CF93BE
:101DB000809178078F5F809378070BE115E0C0E092
:101DC0008C2F80640E94B60E80E80E94B60E61E0FF
:101DD00080917B070E94110380917C0718161CF4E8
:101DE00060E00E94110380E090E0F801E80FF91F25
:101DF00020812EBD00000DB407FEFDCF2EB501964B
:101E00008435910591F780917C0718161CF461E0E8
:101E10000E941103CF5F0C5A1F4FC63089F680E431
:101E2000CF911F910F910C94B60E0F931F93CF93E8
:101E3000DF938C01C0E0D0E0F801EC0FFD1F64914E
:101E4000662371F0E0916C07F0916D070190F081CD
:101E5000E02D8CE697E00995892B11F02196ECCFC7
:101E6000CE01DF91CF911F910F910895CF93DF9312
:101E70000E94150FEC0181E191E00E94230E8C0F6E
:101E80009D1FDF91CF91089588EF91E0EBE1F5E0A0
:101E9000DF019C011D9221503040E1F7109275073F
:101EA0001092760781E694E00E94150F0E94D50EED
:101EB0008CB583608CBD8DB58E7F8DBD84E191E046
:101EC000EEEFFFE30995109272078CE394E00E9415
:101ED000360F0E94D50E0E94620E8091330781302A
:101EE00039F062E370E080E090E00E941804F3CFE4
:101EF0000895AF92BF92CF92DF92EF92FF920F932D
:101F00001F93CF93DF93C82ED12CE601C25ED84F2A
:101F10009DA1992309F44FC07E019FEFE91AF90AA8
:101F2000F70195A1911147C09EA58601000F111FD1
:101F3000025E184FF80134A525A5E32FF22FE90F13
:101F4000F11DE90FF11D259134912F3FFFEF3F0760
:101F500011F41DA230C039ABF601EE0FFF1FE85D92
:101F6000F84F3327220F331F05A0F6A1E02DE20F13
:101F7000F31FA590B49081111AC060E083E497E04C
:101F80000E94C704F801B3AAA2AAF601EE0FFF1F30
:101F9000E05DF84F16A215A281E0F70185A389E064
:101FA0008BAF1EAEFE017B9615A2329615A2299626
:101FB0008DA18F5F8DA3DF91CF911F910F91FF9026
:101FC000EF90DF90CF90BF90AF90089570E0DB016D
:101FD000AA0FBB1FA25EB84FD4962C91D497D5966A
:101FE0009C91D597E22FF92FE80FF11DE80FF11D15
:101FF000259134915F9696963C932E939597F9018F
:102000008591949190914707989F802D1124625E4D
:10201000784FFB01B19685A3F901A591B4914B2F9F
:1020200050E0E82FF0E04E175F0720F4F90125910A
:102030003491832FFB01B296899F802D112485A3B3
:102040000895AF92BF92CF92DF92EF92FF920F93DB
:102050001F93CF93DF93182F062FC1E0D3E08AEFB1
:10206000D82E9EEFE92E842F8470C82E842F827084
:10207000B82E842F8870A82E4170F42E8C2F880FD4
:102080008F5FE80ECC2081F04D2F400F6C2F610F39
:102090008CE697E00E9422054C2F400F6D2F610FB8
:1020A0008CE697E00E942205BB2081F0402F4D1B5B
:1020B0006C2F610F8CE697E00E942205402F4C1B8D
:1020C0006D2F610F8CE697E00E942205AA2081F017
:1020D0004C2F400F612F6D1B8CE697E00E9422056C
:1020E0004D2F400F612F6C1B8CE697E00E9422055C
:1020F000FF2081F0402F4C1B612F6D1B8CE697E079
:102100000E942205402F4D1B612F6C1B8CE697E02F
:102110000E942205CD1744F4E7FC04C0D150D394AB
:10212000D394ED0CCF5FAACFDF91CF911F910F9188
:10213000FF90EF90DF90CF90BF90AF9008959F9267
:10214000AF92BF92CF92DF92EF92FF920F931F93C5
:10215000CF93DF93F82EE62EB22E03E0020FD0E0ED
:10216000C3E08AEFC82E1EEF842F8170982EAA2418
:10217000A394A20E4270D42EDF5F802F8B19180F0C
:102180009920A1F02C2F220F2A0D4E2D4C1B6D2FC4
:102190006F0D8CE697E00E949206202F4E2D4D1B6E
:1021A0006C2F6F0D8CE697E00E949206DD20A1F067
:1021B0002C2F220F2A0D4E2D4C1B6F2D6D1B8CE6E4
:1021C00097E00E949206202F4E2D4D1B6F2D6C1B09
:1021D0008CE697E00E949206DC1744F417FD04C0D9
:1021E000C150C394C3941C0D0E5FC6CFDF91CF9135
:1021F0001F910F91FF90EF90DF90CF90BF90AF9025
:102200009F9008958F929F92AF92BF920F931F93CA
:10221000CF93DF93CDB7DEB7A1970FB6F894DEBFAB
:102220000FBECDBF19A2423008F44AE08E010F5D07
:102230001F4F842E912CA12CB12CA50194010E943A
:10224000E418E62FB901CA0101501109EA3014F46B
:10225000E05D01C0E95CD801EC93232B242B252BF6
:1022600061F7C8010E94230EA1960FB6F894DEBF55
:102270000FBECDBFDF91CF911F910F91BF90AF9057
:102280009F908F900895E0916C07F0916D070190F9
:10229000F081E02D682F8CE697E0099480913A0751
:1022A00090913B07892BB1F1809142078F7169F5BD
:1022B00084E10E94DC03BC01990F880B990B0E94FA
:1022C000461926EE3FE34EEC50E40E94AA190E9404
:1022D00015199B017093390760933807672B91F0AC
:1022E00084E080933707EAE3F7E080E04191519181
:1022F0002417350718F48093370708958F5F8430CB
:10230000A9F703C08FEF80933707809142078F5F53
:102310008093420708958F929F92AF92BF92CF927F
:10232000DF92EF92FF920F931F93CF93DF93FB0106
:1023300024913196C490F0908C07022E000C330B40
:10234000121613060CF0D7C080330CF0D4C0482FFF
:10235000082E000C550BFA01EC0DF11DC7FCFA9587
:102360001E161F060CF0C7C06E5F7F4FD90117966F
:1023700093E0B595A7959A95E1F787FF0BC0C80E36
:10238000A49FC001A59F900DB49F900D1124681BC0
:10239000790B80E04C2D0C2C000C550B480F511D77
:1023A00087FD5A95413351051CF090E3C92EC81A98
:1023B0002535310514F024E530E010917807182711
:1023C000982F977031E001C0330F9A95EAF7859501
:1023D00085958595F4E58F02C0011124855E9A4F9D
:1023E00000E00C2C000CDD08BB24B394402F50E01F
:1023F0004C155D050CF07FC0FB01E490F1E0FF128D
:1024000018C0FB01EC0140E8542F5E2119F05881FF
:10241000532B588350E0559547954115510519F4B4
:102420003196E49040E821965C2F581B521760F3D8
:1024300059C0F1101AC0A32EA094FB01EC0140E892
:10244000542F5E2119F058815A21588350E0559538
:1024500047954115510519F43196E49040E82196CD
:102460005C2F581B521760F33DC043E0F41223C0A9
:10247000932E9094FB01EC0140E8A82E8C2E881A34
:10248000542F5E2141F08126588180FE02C0532BDB
:1024900001C05921588350E0559547954115510584
:1024A00019F43196E49040E821965C2F5A1952179E
:1024B00028F31B2517C0FB01EC0140E8542F5E21D7
:1024C00019F058815327588350E055954795411589
:1024D000510519F43196E49040E821965C2F581B81
:1024E000521760F3330F19F48C5A9F4F31E00F5F8E
:1024F0006A0F7B1F7BCFDF91CF911F910F91FF90D0
:10250000EF90DF90CF90BF90AF909F908F90089505
:10251000CF93DF93CDB7DEB762970FB6F894DEBFE7
:102520000FBECDBF789484B5826084BD84B58160D0
:1025300084BD85B5826085BD85B5816085BD80918E
:102540006E00816080936E00109281008091810006
:1025500082608093810080918100816080938100FE
:10256000809180008160809380008091B1008460C0
:102570008093B1008091B00081608093B000809121
:102580007A00846080937A0080917A0082608093E0
:102590007A0080917A00816080937A0080917A003D
:1025A000806880937A001092C10082E380939D0737
:1025B00081E090E0A0E0B0E08093990790939A07C3
:1025C000A0939B07B0939C078FEF80938E07E0E862
:1025D000F7E7259134912130304C09F049C0E6E904
:1025E000F7E7E491E0937707E7E9F7E7E491E09311
:1025F0002207E8E9F7E7E491E0932307E9E9F7E741
:10260000859194919093250780932407EBE9F7E750
:1026100085919491909327078093260788E0809373
:102620004907EEE9F7E7E491E0934807EFE9F7E7B8
:10263000E491E0938E07E0EAF7E785919491909317
:102640003B0780933A07E2EAF7E7859194919093EC
:102650003D0780933C07E4EAF7E7859194919093D6
:102660003F0780933E07E6EAF7E7859194912CC0F7
:102670009CE390937707109222078093230780E2D0
:1026800093E0909325078093240784ED93E0909343
:1026900027078093260788E080934907809348079F
:1026A0008CEA9DE090933B0780933A078EED9DE086
:1026B00090933D0780933C0784E79EE090933F070B
:1026C00080933E078CE39FE09093410780934007FF
:1026D00011E010931E076FEF70E085E00E947D030C
:1026E00088E08093280789E08093290787E080931A
:1026F0002A0786E080932B0704E000932C0782E0F2
:1027000080932D0781E180932E070E94620E8CE357
:102710009FE0909339078093380700933707109311
:1027200042078BE080937A078DE08093790780E100
:1027300080937B078EE080937D078FE080937C07FA
:102740001093740710938C0710928D0710937307E2
:10275000E6EAF2E0E491EF5FE0937007E7EAF2E087
:10276000E491EF5FE093710788EA92E090938B0722
:1027700080938A071FB7F8948091D104811127C0F4
:10278000EDE9F4E08491E1EBF4E09491E82FF0E0DE
:10279000EE0FFF1FEC58FF4FA591B491EC91E92388
:1027A00021F461E08AE00E94110361E08AE00E9466
:1027B00041038CB580618CBD8CB580648CBD61E0BB
:1027C0008DE00E94410361E08BE00E944103809113
:1027D000D1048F5F8093D1041FBF8CB58F7D8CBDDA
:1027E0008CB58C7F81608CBD8DB581608DBD8CB5C5
:1027F0008C608CBD61E080917A070E94410361E0AA
:10280000809179070E94410361E080917B070E94DB
:10281000410380917D0718161CF461E00E9441037A
:1028200080917C0718161CF461E00E94410380919E
:102830007D07181674F460E00E9411036AE070E0EE
:1028400080E090E00E94180461E080917D070E9482
:10285000110380917907082E000C990BFC01ED56AD
:10286000FB4FE491F0E0EE0FFF1FE258FF4F259180
:1028700034913093810720938007FC01E955FB4F89
:10288000E491E093870780917A07082E000C990B5A
:10289000FC01ED56FB4FE491F0E0EE0FFF1FE25814
:1028A000FF4F2591349130937F0720937E07FC01E1
:1028B000E955FB4FE491E093860780917C07082E51
:1028C000000C990BFC01ED56FB4FE491F0E0EE0F8C
:1028D000FF1FE258FF4F25913491309383072093D7
:1028E0008207FC01E955FB4FE491E0938807809152
:1028F0007B07082E000C990BFC01ED56FB4FE49171
:10290000F0E0EE0FFF1FE258FF4F25913491309316
:10291000850720938407FC01E955FB4FE491E09380
:10292000890781E20E94B60E84E10E94B60E809172
:10293000770787FF03C08FE780937707809177073A
:1029400080680E94B60E80E20E94B60E8CE00E9463
:10295000B60E0E94D50E11E01093470784E08093D5
:102960006B0780E790E0909353078093520760E0F5
:1029700080E00E94E60F61E070E083E00E947D034A
:102980008091B100887F81608093B100F8941092AB
:10299000800010928100109285001092840088E1DE
:1029A00091E09093890080938800809181008860F5
:1029B000809381008091810081608093810080916B
:1029C0006F00826080936F0078940E944E11809116
:1029D0003407813019F4109248071EC080913707E0
:1029E0008823C9F360E083E497E00E94C70488E885
:1029F00090E09093510780935007109256071092E1
:102A000055071093440789E08093590710925C079B
:102A100010925E07109260070E94B70811E00E94B2
:102A2000D609882309F479C280913507813009F4E9
:102A30007CC28091CF049091D004892B09F0ABC067
:102A40008091CD049091CE04892B09F0A4C000910F
:102A5000CA04A02EB12CC50102972091CB0430915D
:102A6000CC042817390769F5D090C704ED2CF12C58
:102A70009701225031094091C8045091C90442176E
:102A80005307F9F486E990E09093A3078093A20797
:102A900098E49093A40783E497E00E94A70428E2B7
:102AA000E216F1041CF46AE06D0D01C062E338E245
:102AB000A316B1041CF48AE0800F01C082E30E94D7
:102AC0007B078091300781508E3F90F4E090C804DE
:102AD000F090C9041E141F045CF40091CB04402F35
:102AE0006E2D8EE893E00E94E406882309F420C24C
:102AF0008091320781508E3FC8F4C090C804D090B6
:102B0000C9048091C70490E00297C816D90674F4EE
:102B10000091CB04FF24F394FC0C402F6F2D8EE822
:102B200093E00E94E406882309F420C280912F07D5
:102B300081508E3F90F4E090CB04F090CC041E14B2
:102B40001F045CF40091C8044E2D602F8CE191E0CD
:102B50000E94E406882309F428C28091310781503D
:102B60008E3FC8F4C090CB04D090CC048091CA04AE
:102B700090E00297C816D90674F4FF24F394FC0C75
:102B80000091C8044F2D602F8CE191E00E94E40673
:102B9000882309F42EC210938C0710938D0720917F
:102BA000C8043091C9043A8B298B263031052CF0AA
:102BB000590136E0A31AB10802C0A12CB12C95012D
:102BC00049895A89241B350B56E0529FC001539FF7
:102BD000900D1124212C312C29893A892B5F3F4FEC
:102BE0003D872C87AC014C5E5F4F5F874E87C0905E
:102BF000C704D12CAC14BD044CF0E090CF04F0908D
:102C0000D0041E141F040CF4D2C0E9C08C859D852D
:102C10008A159B0594F38091CB049091CC04893064
:102C200091052CF07C0159E0E51AF10802C0E12C75
:102C3000F12C2E853F85220D331D3E832D83A70168
:102C4000481B590B66E0649F9001659F300D11246D
:102C5000412C512CAC01485F5F4F58874F83C9010D
:102C600086969A8789879A2C9601215031093C8350
:102C70002B833FEF3A0D3B878091CA0490E0E81622
:102C8000F9060CF08DC04F8158854E155F050CF488
:102C900087C0C090CF04D090D00429853A85240DF8
:102CA000351DC20ED31E6090CD047090CE044D81B0
:102CB0005E81640E751E0197E816F9060CF055C08A
:102CC0008E2C4E2D692D8EE893E00E94E406882319
:102CD00039F027E0462D6C2D8CE697E00E947A05AE
:102CE0008B819C81A816B9060CF03FC0482D692D38
:102CF00085E592E00E94E4068823B9F132E0360DC2
:102D0000398352E05C0D5A8303E023E0432F652FA3
:102D10008CE697E00E949D051A141B048CF4482D44
:102D20006B8585E592E00E94E406882349F0482DF2
:102D3000692D8EE893E00E94E406882309F476C1A9
:102D40001E141F0494F44FEF480D692D85E592E0A1
:102D50000E94E406882349F0482D692D8CE191E01A
:102D60000E94E406882309F46BC18B819C81A8161C
:102D7000B9067CF44E2D692D8CE191E00E94E406A9
:102D8000882339F027E0462D6C2D8CE697E00E94D1
:102D900092069FEFE91AF90A26E0420E511C6CCF09
:102DA0005FEFA51AB50A66E0260E311C20CF4091D0
:102DB000CB045091CC0414161506ACF5415069892A
:102DC00085E592E00E94E406882369F110928C0761
:102DD00010928D0703E02E2D46E16BE22CC0E1142A
:102DE000F10469F14091CB045091CC048091CA0464
:102DF00090E002972E2D2195481759070CF02AC113
:102E00004F5F698985E592E0288B0E94E406288956
:102E1000882309F41FC110928C0710928D0703E0DC
:102E200046E168E21EC110938C0710938D0703E002
:102E30002E2D46E168E28CE697E00E949D05A09069
:102E4000CD04B090CE041A141B04CCF429893A891D
:102E5000121613060CF007C1622F61504091CB048B
:102E600085E592E00E94E406882309F4FCC01092F4
:102E70008C0710928D070A2D23E049E1FBC0A114B5
:102E8000B10409F405C132E0C31AD1080A2D019535
:102E900049895A894C155D058CF4642F6F5F409108
:102EA000CB0485E592E00E94E406882339F0109275
:102EB0008C0710928D0723E046E106C010938C0723
:102EC00010938D0723E049E14A0D68E28CE697E014
:102ED0000E949D05F7FED4C05FEFE51AF50AF09257
:102EE000D004E092CF04B7FCCBC08091CF04909186
:102EF000D004181619062CF401979093D0048093EF
:102F0000CF048091CD049091CE04181619062CF4AC
:102F100001979093CE048093CD0480E090E0892BBC
:102F200009F47DCD0E94000079CD0E94B70881CDC3
:102F3000402F6FEF6E0D85E592E00E94E406882336
:102F400039F020E0402F6E2D85E592E00E94B50615
:102F5000B701615071097093C9046093C8044AEFC6
:102F60005FEF5093CE044093CD041CC0402F6F2DD3
:102F700085E592E00E94E406882339F020E0402FA6
:102F80006C2D85E592E00E94B506B6016F5F7F4F1C
:102F90007093C9046093C80486E090E09093CE04D7
:102FA0008093CD0421E0402F1FC04FEF4E0D602FC6
:102FB00085E592E00E94E406882339F020E04E2D5A
:102FC000602F85E592E00E94B506A70141505109A6
:102FD0005093CC044093CB042AEF3FEF3093D004BE
:102FE0002093CF0421E0602F85E592E00E94B50692
:102FF000D2CD4F2D602F85E592E00E94E406882314
:1030000039F020E04C2D602F85E592E00E94B50656
:10301000A6014F5F5F4F5093CC044093CB0486E0F2
:1030200090E09093D0048093CF04DCCF03E023E0C2
:103030004FEF460D6A818CE697E00E949D0580CE99
:1030400003E023E049816FEF6C0D8CE697E00E946E
:103050009D058BCE10938C0710938D0703E046E1FE
:103060006BE26E0DE8CE10938C0710938D070A2D3E
:1030700023E046E168E28CE697E00E949D0508C0E7
:103080006FEFA61AB60AB092CE04A092CD042DCF4F
:10309000F7FE2BCF21CF10926F0710926E0789E0B9
:1030A00091E090936D0780936C0708958F929F92A3
:1030B000AF92BF92CF92DF92EF92FF92CF93DF93C6
:1030C000EC01688179818A819B8161157105810597
:1030D000910521F464E279ED8BE597E02DE133EF82
:1030E00041E050E00E94B21849015A019B01AC0135
:1030F000A7EAB1E40E94D1186B017C01ACEEB4EFF9
:10310000A50194010E94DF18DC01CB018C0D9D1DEF
:10311000AE1DBF1DB7FF03C00197A109B04888834A
:103120009983AA83BB83BC01CD019F77DF91CF91A7
:10313000FF90EF90DF90CF90BF90AF909F908F90D7
:1031400008950E945618089581E091E00E94561853
:10315000089560930101709302018093030190939D
:1031600004010895052E97FB1EF400940E94C918CF
:1031700057FD07D00E94E41807FC03D04EF40C94CE
:10318000C91850954095309521953F4F4F4F5F4F4F
:10319000089590958095709561957F4F8F4F9F4FC3
:1031A00008950E940619A59F900DB49F900DA49FAD
:1031B000800D911D11240895B7FF0C94D1180E9421
:1031C000D118821B930B0895A1E21A2EAA1BBB1BD8
:1031D000FD010DC0AA1FBB1FEE1FFF1FA217B307E3
:1031E000E407F50720F0A21BB30BE40BF50B661FF9
:1031F000771F881F991F1A9469F7609570958095BD
:1032000090959B01AC01BD01CF010895A29FB00133
:10321000B39FC001A39F700D811D1124911DB29F0A
:10322000700D811D1124911D08950E94891988F047
:103230009F5798F0B92F9927B751B0F0E1F0660F7A
:10324000771F881F991F1AF0BA95C9F714C0B130BB
:1032500091F00E94A319B1E008950C94A319672F6F
:10326000782F8827B85F39F0B93FCCF386957795EA
:103270006795B395D9F73EF49095809570956195D3
:103280007F4F8F4F9F4F0895E89409C097FB3EF4FE
:1032900090958095709561957F4F8F4F9F4F9923A3
:1032A000A9F0F92F96E9BB279395F6958795779521
:1032B0006795B795F111F8CFFAF4BB0F11F460FFE1
:1032C0001BC06F5F7F4F8F4F9F4F16C0882311F039
:1032D00096E911C0772321F09EE8872F762F05C04D
:1032E000662371F096E8862F70E060E02AF09A95E8
:1032F000660F771F881FDAF7880F9695879597F9DD
:10330000089557FD9058440F551F59F05F3F71F0D5
:103310004795880F97FB991F61F09F3F79F087953C
:103320000895121613061406551FF2CF4695F1DFC5
:1033300008C0161617061806991FF1CF8695710555
:10334000610508940895E894BB2766277727CB0189
:1033500097F908950E94BD190C942E1A0E94201A04
:1033600038F00E94271A20F0952311F00C94171AB8
:103370000C941D1A11240C94A4190E94811970F345
:10338000959FC1F3950F50E0551F629FF001729F0A
:10339000BB27F00DB11D639FAA27F00DB11DAA1F19
:1033A000649F6627B00DA11D661F829F2227B00D66
:1033B000A11D621F739FB00DA11D621F839FA00DF1
:1033C000611D221F749F3327A00D611D231F849F41
:1033D000600D211D822F762F6A2F11249F57504098
:1033E0009AF0F1F088234AF0EE0FFF1FBB1F661F13
:1033F000771F881F91505040A9F79E3F510580F0DC
:103400000C94171A0C94A4195F3FE4F3983ED4F37C
:10341000869577956795B795F795E7959F5FC1F77F
:10342000FE2B880F911D9695879597F9089597F92A
:103430009F6780E870E060E008959FEF80EC08955A
:1034400000240A9416161706180609060895002483
:103450000A9412161306140605060895092E0394FD
:10346000000C11F4882352F0BB0F40F4BF2B11F471
:1034700060FF04C06F5F7F4F8F4F9F4F0895DB0148
:103480008F939F930E94D118BF91AF91A29F800DFF
:10349000911DA39F900DB29F900D11240895991B2B
:1034A00079E004C0991F961708F0961B881F7A953B
:1034B000C9F78095089597FB072E16F4009407D05E
:1034C00077FD09D00E946F1A07FC05D03EF4909555
:1034D00081959F4F0895709561957F4F0895AA1B20
:1034E000BB1B51E107C0AA1FBB1FA617B70710F0EF
:1034F000A61BB70B881F991F5A95A9F78095909521
:10350000BC01CD010895EE0FFF1F0590F491E02D51
:10351000099481E090E0F8940C948E1AF894FFCF0F
:10352000010100000000000000C6059602E302E26F
:0C353000020D0A004C4F414445520000BF
:00000001FF
